:020000040000FA
:04000000D2303A2898
:08000800A000030EA100831209
:1000100005191028831601178312B23081002B288E
:1000200083160113831203140B190310A80DA90DD5
:10003000AA0DAB0DAC0DAC16FF302C02031D2B2806
:10004000FA302B02031D2B2831152A08AF0029088E
:10005000AE002808AD008B100B11210E8300A00EFE
:04006000200E090065
:0C007400203084008001840A80300402E7
:10008000031C3C281230B0005921850187018316DA
:100090000C30850587018312831605148715071612
:1000A0008312850187010730990000309A001030D3
:1000B00083168E008312603083168F008312003007
:1000C000831691009F008312C8308316810083122B
:1000D00031309000003083168C00831210308B007A
:1000E000851D0027BB2181018E018F010B118B1013
:1000F0000B108C018B178A2031198D20B30B8828A7
:10010000031085190314B90DF03039020319E620E4
:10011000C0237B2864003210080031110130B70081
:100120008B132030370783169B001C141A08831288
:10013000A4001030370783169B001C141A08831282
:10014000A300A6000230A6060030370783169B00E6
:100150001C141A088312A200A7000130A7068B17EF
:10016000321CB82822090339A200A309A409A50951
:1001700024082F02031DE02823082E02031DE02877
:1001800022082D02031DE02801303702031DCB2871
:100190003D143E149B2102303702031DD228BD14AA
:1001A0003E149F2103303702031DD9283D153E140C
:1001B000A32104303702031DE028BD153E14A721FA
:1001C000B70A053037020318080090283C1C0800C5
:1001D0000130B600B300B400B500B7008501870157
:1001E000B1138A20B30B0A29031085190314B90D22
:1001F000F030390203193129B41F0710B40B0A2952
:100200003708B6080319B600031908290714B603FE
:100210009630B400311DF1283111321C14292D09FA
:100220000339AD00AE09AF092F1CF1288E018F01F3
:100230000C1CF1280C102E1EF1288B1320303707D0
:10024000BB002F08BA00442110303707BB002E082E
:10025000BA00442100303707BB002D08BA00442102
:100260008B1785018701B70AB60105303702031CD9
:10027000F128BB2108003E1C08003E101030BB00D6
:100280003D08BA00442108008B133A0883161C1558
:100290009A0083123B0883169B0055309D00AA30BC
:1002A0009D009C1464009C1852291C1183128B170A
:1002B0000800831600309B001C141A088312BC002F
:1002C000831610309B001C141A088312BD000030E6
:1002D0009500603084008B13831604089B001C1467
:1002E0001A0883128B178000840A68300402031CEA
:1002F0006B296430D5003F24DC003C30EC00ED007D
:10030000EE00EF00EA146E30D5003F240F39031DD4
:10031000080044240F39031D080049240F39031D28
:1003200008004E240F39031D080083168711071299
:100330008312EA1008000130E800CA2108000230E8
:10034000E800CA2108000430E800CA21080008308B
:10035000E800CA2108001030E800CA210800203057
:10036000E800CA2108004030E800CA2108008030B7
:10037000E800CA210800EA178B13831670309B002F
:100380001C141A0883128B17E800CA210430EB00F2
:10039000EA130800E80803190800681CD729673029
:1003A000D5003F24D1006830D5003F24D200E81C9E
:1003B000E1296730D5004424D1006830D5004424B9
:1003C000D200681DEB296730D5004924D100683080
:1003D000D5004924D200E81DF5296730D5004E2408
:1003E000D1006830D5004E24D200681EFF296A3043
:1003F000D5003F24D1006B30D5003F24D200E81E49
:10040000092A6A30D5004424D1006B30D500442439
:10041000D200681F132A6A30D5004924D1006B30FE
:10042000D5004924D200E81F1D2A6A30D5004E2489
:10043000D1006B30D5004E24D200EA16D11A2D2AF5
:10044000511B2D2A511C2D2ADC1FEA125C1F2D2A5C
:10045000501C2D2AC01B2D2A0800EA1E3D2AEA1B2B
:100460003D2A511870308B1383169B001C141A08F8
:1004700083128B17680203190800D11A482A511BEE
:10048000482A6A10511C482A5014051E6A14051681
:10049000511C502A511A5016D11AC017511B501214
:1004A000EA1F572AD11A0800511B08005B2AD11AEB
:1004B000882A511B882A6530D500521A3F24D21A47
:1004C0004424521B4924D21B4E245118C4006630C8
:1004D000D500521A3F24D21A4424521B4924D21B5D
:1004E0004E245118CC0052085118D70004306A1815
:1004F0003230EA1B32305118C80051185C14EA1F20
:10050000862A511C852A4403C00008005118C001E6
:1005100051187030BB006808E900BA004421BD01E1
:100520000800FD010730FF007B08FE0C03189C2A21
:10053000FF0B952AFB0100340310A12AFE0C0318BF
:10054000FB07FB0CFD0CFF0B9E2AFB0CFD0C003483
:1005500094019301093095008B138E018F018B1745
:10056000D6135608FB007508F51BFF3CFE00FE1372
:100570009122FD0D7B0DF51FD607F51BD6025608FF
:0E058000760793000318141408309500080045
:1007800002300F02031C0800EA1CE82BA127F10825
:100790000319E82B6E30D50071183F24F11844245A
:1007A000E80068189B21E8189F216819A321E8191F
:1007B000A7216E30D50071194924F1194E24E800A3
:1007C00068189B21E8189F216819A321E819A7211F
:1007D0000730EB0503308A006B088207F32B2A2CC5
:1007E0002B2C2C2C2D2C501C382C4008D500571AA3
:1007F0003F24D71A4424571B4924D71B4E24D60024
:100800006108F5006008F6005C1CA822C80B382CB3
:100810004C085C180530C8005C1CC00A5C10440819
:100820004002031C382CC01B192C501E192CC0016F
:10083000382C7A18202C7A140930C800C003382CC0
:100840005012DC1805125C1950105C1DC0035C1DB1
:10085000C017382C382C382C382C071C312C07109A
:10086000382CE9080319382C07140310E90C382C2C
:10087000EB0A05306B020318EB018F01080005300D
:100880008A00D5135508820005308A00D51755080F
:10089000820006308A00D5135508820006308A008F
:0608A000D5175508820087
:100A00000034013403340434053406340834093422
:100A10000A340B340D340E340F34113412341334C1
:100A2000143416341734183419341B341C341D3460
:100A30001E342034213422342434253426342734FF
:100A400029342A342B342C342E342F34303432349D
:100A50003334343435343734383439343A343C343C
:100A60003D343E34403441344234433445344634DA
:100A7000473448344A344B344C344D344F3450347A
:100A800051345334543455345634583459345A3418
:100A90005B345D345E345F346134623463346434B7
:100AA00066346734683469346B346C346D346E3456
:100AB00070347134723474347534763478347A34F2
:100AC0007B347D347F347F34C43464340134013466
:100AD0001134003401341134003400340134003452
:100AE0000034003400340034003400340034003466
:100AF0000034003400340034003400340034003456
:100B00007F347E347C347B347A3479347734763471
:100B1000753474347234713470346E346D346C34B2
:100B20006B346934683467346634643463346234F3
:100B300061345F345E345D345B345A345934583434
:100B40005634553454345334513450344F344D3476
:100B50004C344B344A3448344734463445344334B7
:100B6000423441343F343E343D343C343A343934F9
:100B700038343734353434343334323430342F3439
:100B80002E342C342B342A3429342734263425347B
:100B900024342234213420341E341D341C341B34BC
:100BA00019341834173416341434133412341134FD
:100BB0000F340E340D340B340A3409340634053442
:100BC0000434033401340034C43464340134013453
:100BD0002234003401342234003400340034003430
:100BE0000034003400340034003400340034003465
:100BF0000034003400340034003400340034003455
:100C000080340034003401340234033404340634B4
:100C100008340A340C340E341134143417341A34B2
:100C20001D342134243428342C342F3433343734D5
:100C30003B343F34433447344B344F3452345634CE
:100C40005A345D346134643467346A346D347034DA
:100C500072347434763478347A347B347C347D3432
:100C60007E347E347E347E347E347D347C347B34FA
:100C70007A34783476347434723470346D346A343F
:100C80006734643461345D345A34563452344F34EA
:100C90004B34473443343F343B34373433342F34CC
:100CA0002C342834243421341D341A3417341434A9
:100CB00011340E340C340A3408340634043403344A
:100CC0000234013400340034C43464340134113447
:100CD00044340034013444340034003402340034E9
:100CE0000034003400340034003400340034003464
:100CF0000034003400340034003400340034003454
:100D000080340034003401340234033404340634B3
:100D100008340A340C340E341134143417341A34B1
:100D20001D342134243428342C342F3433343734D4
:100D30003B343F34433447344B344F3452345634CD
:100D40005A345D346134643467346A346D347034D9
:100D500072347434763478347A347B347C347D3431
:100D60007E347E347E347E347E347D347C347B34F9
:100D70007A34783476347434723470346D346A343E
:100D80006734643461345D345A34563452344F34E9
:100D90004B34473443343F343B34373433342F34CB
:100DA0002C342834243421341D341A3417341434A8
:100DB00011340E340C340A34083406340434033449
:100DC0000234013400340034C43464340134413416
:100DD0008834003401348834003400340034003462
:100DE0000034003400340034003400340034003463
:100DF0000034003400340034003400340034003453
:100E00003C1C08006C146D14EB011430B600071084
:100E10000130EB0507308A006B088207102F172F6F
:100E20006108F5006008F6000516D6011A2F7F301C
:100E3000D6001A2F701A432F6B18232F7019F60A39
:100E40007018F603272F7019F50A7018F503503043
:100E50007018EC007019ED00C8307602C830031825
:100E6000F600503076025030031CF600F51F3E2F7E
:100E7000A0307502A030031CF500432F64307502CA
:100E800064300318F5007F30D6006B1CD601A82211
:100E9000EA017927701C4E2F6D1B7016701D522FA2
:100EA0006C1B7016701E572FEB0A6B1C682F0710F7
:100EB000B60B5F2F07143C306B180A30B600640085
:100EC0000A300F02031C5F2F8F01701A082F1A2F90
:100ED0007508E1007608E000603084000408BB007B
:100EE0000008BA004421840A68300402031C6E2FF3
:100EF0000800F0010A30851DEC078519EC027830F6
:100F00006C020319701479300318EC0015306C0270
:100F10000319F0141430031CEC000A30051CED0713
:100F20000518ED0278306D02031970157930031839
:100F3000ED0015306D020319F0151430031CED009F
:100F40000800F10114308719EE070230871DEE0208
:100F5000EE1BB42F14306E020318BC2F1430EE00B9
:100F6000F21CF1147210BC2F721C7114F2106E1B63
:100F7000BA2FBC2FC030EE001430071AEF07023032
:100F8000071EEF02EF1BCE2F14306F020318D62F6F
:100F90001430EF00F21DF1157211D62F721D71156C
:0E0FA000F2116F1BD42FD62FC030EF000800C7
:084000000A00030005000200A4
:02400E00CC33B1
:10420000010078007A007C007E007B0079007F004E
:104210007D007A0078007E007C00FF00FF00FF0038
:104220000000F200F600FA00FE00F200F600FA00CC
:10423000FE00F200F600FA00FE00FF00FF00FF00A3
:10424000010005000500050005000900090009003E
:1042500009000D000D000D000D00FF00FF00FF0024
:10426000FF00FF00FF00FF00FF00FF00FF00FF0056
:10427000FF00FF00FF00FF00FF00FF00FF00FF0046
:10428000FF00FF00FF00FF00FF00FF00FF00FF0036
:10429000FF00FF00FF00FF00FF00FF00FF00FF0026
:1042A000FF00FF00FF00FF00FF00FF00FF00FF0016
:1042B000FF00FF00FF00FF00FF00FF00FF00FF0006
:1042C0007D00FC007D00FC007D00FC007D00FC000A
:1042D000FF00FF00FF00FF00FF00FF00FF00FF00E6
:1042E0000000000000000000FF00FF00FF00FF00D2
:1042F000FF00FF00FF00FF00FF00FF00FF00AA001B
:00000001FF
